:100000000C9464000C948C000C948C000C948C0068
:100010000C949A000C948C000C948C000C948C0022
:100020000C948C000C948C000C948C000C944D0B54
:100030000C948C000C948C000C948C000C948C0010
:100040000C947E0C0C948C000C94D0100C941E110B
:100050000C948C000C948C000C948C000C948C00F0
:100060000C948C000C948C000000000024002700ED
:100070002A0000000000250028002B0000000000DE
:1000800023002600290004040404040404040202DA
:100090000202020203030303030301020408102007
:1000A0004080010204081020010204081020000012
:1000B0000007000201000003040600000000000029
:1000C00000008E0086078A1211241FBECFEFD8E0F1
:1000D000DEBFCDBF11E0A0E0B1E0ECE2FBE202C088
:1000E00005900D92A838B107D9F713E0A8E8B1E060
:1000F00001C01D92A337B107E1F710E0C8ECD0E0D2
:1001000004C02297FE010E949015C23CD107C9F796
:100110000E9477100C9494150C94000088E891E0EC
:100120000E94D909089581E593E060E071E00E94A2
:10013000641008951F920F920FB60F921124EF9240
:10014000FF920F931F932F933F934F935F936F9360
:100150007F938F939F93AF93BF93EF93FF93809180
:100160006502882309F445C08EE00E94FB0D892BAF
:1001700021F481E0809362023CC080916202882376
:10018000C1F1109262028091630290916402019623
:1001900090936402809363020E94C60C0E94E21353
:1001A00020E030E040E85CE30E9498140E94B6131F
:1001B0009B01AC018091660290916702A091680258
:1001C000B091690279018A01E81AF90A0A0B1B0B3E
:1001D000D801C7014A97A105B10518F081E08093C5
:1001E0006A0220936602309367024093680250933C
:1001F0006902FF91EF91BF91AF919F918F917F9194
:100200006F915F914F913F912F911F910F91FF90AF
:10021000EF900F900FBE0F901F90189583E060E055
:1002200070E00E941E0C8BE060E070E00E941E0CEB
:10023000809176018823D9F480918B0190918C0173
:10024000A0918D01B0918E0180936E0290936F0208
:10025000A0937002B093710281E080936D021092BE
:1002600093011092940110929501109296010895B5
:10027000AF92BF92CF92DF92EF92FF920F931F93B4
:10028000CF93DF93C0916B02D0916C02CE010197A6
:10029000029758F00F2EF0E0AF2EF0E0BF2EF0E006
:1002A000CF2EF0E0DF2EF02D18C060916302709128
:1002B0006402882777FD8095982F0E94E41320E040
:1002C00030E044E353E40E9449135B016C01229740
:1002D00021F4D7FAD094D7F8D094109264021092F7
:1002E0006302E090DA01F090DB010091DC011091F3
:1002F000DD0180E090E0A0E0B0E08093DA0190932F
:10030000DB01A093DC01B093DD0181E593E060E1C6
:1003100071E00E947A0F81E593E0B601A50122E029
:1003200030E00E94611081E593E068E171E00E9495
:100330007A0F81E593E0B801A70122E030E00E9446
:10034000611081E593E06AE171E00E946410DF9141
:10035000CF911F910F91FF90EF90DF90CF90BF90C2
:10036000AF9008950E94380181E593E06CE171E05F
:100370000E94641010926D0281E0809376011092C9
:100380006C0210926B0280918B0190918C01A09174
:100390008D01B0918E018093DE019093DF01A093D7
:1003A000E001B093E1010895CF92DF92EF92FF92C6
:1003B0000F931F93DF93CF93CDB7DEB7CE57D040C7
:1003C0000FB6F894DEBF0FBECDBF8E010F5F1F4F7B
:1003D00078018FE7C82ED12CCC0EDD1E87E792E086
:1003E00068E570E04EE350E021E030E00E949609BD
:1003F00087E792E00E947207D7018D937D01AC15CB
:10040000BD0561F7E4EEF1E0D8013C9120E01196E2
:100410008C9190E0822B932B819391930E5F1F4FD1
:100420000E151F0589F7C258DF4F0FB6F894DEBFCF
:100430000FBECDBFCF91DF911F910F91FF90EF9035
:10044000DF90CF9008950F931F9307E712E0C80144
:1004500068E570E04DE350E021E030E00E9496094D
:10046000C8010E94720790E09695879596958795AA
:1004700081701F910F9108951F9387E792E068E5BF
:1004800070E042E250E021E030E00E94960987E708
:1004900092E00E947207882381F387E792E068E583
:1004A00070E047E250E022E030E00E94960987E7E2
:1004B00092E00E947207182F87E792E00E9472076D
:1004C000512F40E0282F30E0242B352BC9011F91FC
:1004D000089585E060E070E00E941E0C86E060E018
:1004E00070E00E941E0C83E060E070E00E941E0C31
:1004F0008BE060E070E00E941E0C88E891E00E94B2
:10050000F30908951F93CF93DF9380919701909102
:1005100098018137910571F46091990170919A0168
:1005200085E00E941E0C8CE060E00E94A70D89E02F
:1005300061E010C08F36910581F46091990170914E
:100540009A0185E00E941E0C8CE061E00E94A70DDC
:1005500089E060E00E94A70D07C28037910541F451
:100560006091990170919A0186E00E941E0CFCC175
:100570008637910579F488E891E06AE070E00E949E
:10058000460B6091990170919A0188E891E00E9470
:100590005F0AEAC18737910529F488E891E00E9453
:1005A000F309E2C18D36910549F48FEB92E060E0EA
:1005B00070E0409199010E94120CD6C186369105D7
:1005C000B1F08236910599F08C36910581F0823731
:1005D000910569F08A37910551F08536910539F01A
:1005E0008437910521F08537910509F00CC16091A0
:1005F000990170919A0183E00E941E0C60919B0109
:1006000070919C018BE00E941E0C8091970190914B
:10061000980186369105B9F482E061E00E94A70D49
:1006200084E060E00E94A70D87E060E00E94A70DD3
:1006300088E061E00E94A70D10926D021092760191
:1006400081E090E019C082369105D9F482E060E043
:100650000E94A70D84E061E00E94A70D87E061E0A1
:100660000E94A70D88E060E00E94A70D10926D0225
:100670001092760182E090E090936C0280936B027E
:1006800073C18C369105B9F482E060E00E94A70D39
:1006900084E061E00E94A70D87E060E00E94A70D62
:1006A00088E061E00E94A70D10926D021092760121
:1006B00083E090E0E1CF82379105B9F482E061E018
:1006C0000E94A70D84E060E00E94A70D87E061E032
:1006D0000E94A70D88E060E00E94A70D10926D02B5
:1006E0001092760184E090E0C7CF8A379105B9F483
:1006F00082E060E00E94A70D84E061E00E94A70D07
:1007000087E060E00E94A70D88E061E00E94A70DED
:1007100010926D021092760183E090E019C0853648
:100720009105E1F582E061E00E94A70D84E060E0C0
:100730000E94A70D87E061E00E94A70D88E060E0BD
:100740000E94A70D10926D021092760184E090E055
:1007500090936C0280936B0290919D0180E02091B8
:100760009F013091A001822B932BAA2797FDA09582
:10077000BA2F20918B0130918C0140918D015091C5
:100780008E01820F931FA41FB51F80939301909336
:100790009401A0939501B0939601E6C0843791052A
:1007A000B9F482E061E00E94A70D84E060E00E945D
:1007B000A70D87E060E00E94A70D88E061E00E943D
:1007C000A70D10926D021092760181E090E0C0CFEB
:1007D0008537910509F0C8C082E060E00E94A70D4E
:1007E00084E061E00E94A70D87E061E00E94A70D10
:1007F00088E060E00E94A70D10926D0210927601D1
:1008000082E090E0A5CF8337910519F40E940E0194
:10081000ABC08836910549F582E060E00E94A70DE3
:1008200084E060E00E94A70D87E060E00E94A70DD1
:1008300088E060E00E94A70D80917601882309F08E
:1008400093C080918B0190918C01A0918D01B0910A
:100850008E0180936E0290936F02A0937002B0930A
:10086000710281E080936D027FC08837910529F481
:1008700081E593E063E271E075C08937910519F471
:100880000E94930071C08336910529F481E593E0BD
:100890006EE271E067C08936910511F5109262022F
:1008A000109264021092630221E02093650220936B
:1008B000D90180E090E0A0E0B0E08093DA0190936D
:1008C000DB01A093DC01B093DD0110926A0210926B
:1008D0006D022093760110926C0210926B0244C05C
:1008E0008A36910549F40E943801109265021092EF
:1008F00062021092D90138C08B36910519F40E941A
:10090000380132C08833910591F4C0E0D0E08FEB1C
:1009100092E0BE0140E00E94120C219682E0C030BD
:10092000D807A9F781E593E06FE271E01BC0C99792
:10093000D9F48FEB92E060E070E00E940B0C182F6E
:1009400081E593E06FE371E00E947A0F81E593E027
:10095000612F70E04AE050E00E94670F81E593E06C
:100960006AE171E00E946410DF91CF911F910895B8
:1009700081E593E00E9411129C018D30910519F0E0
:100980008A30910571F48091D7019091D8011816A1
:100990001906BCF40E9482021092D8011092D7016D
:1009A00008958091D7019091D801FC01EE0FFF1FAF
:1009B000E956FE4F3183208301969093D8018093AE
:1009C000D70108958F929F92AF92BF92CF92DF92FC
:1009D000EF92FF920F931F93CF93DF930E94C60C69
:1009E0000E94E21320E030E040E85CE30E949814AB
:1009F0000E94B61360938B0170938C0180938D01DC
:100A000090938E018091D901882309F487C0809149
:100A10007601882309F082C00E942302882309F40A
:100A20007DC00E94D40180916D02882321F18091C4
:100A30006B0290916C0203970297E8F4BB248091BB
:100A40008B0190918C01A0918D01B0918E0120912C
:100A50008F01309190014091910150919201821B40
:100A6000930BA40BB50B81359105A105B10520F0C1
:100A7000BB24B39401C0BB248090E2019090E301B9
:100A8000C090DA01D090DB01E090DC01F090DD0154
:100A9000C4EED1E0AA2408811981080D191DB801FE
:100AA000882777FD8095982F0E94E41320E030E09E
:100AB0004AE753E40E94981420E03EEF4FEF56ECD3
:100AC0000E9449139B01AC010E94E11220E030E03A
:100AD0004AE754E40E9449139B01AC01C701B601E7
:100AE0000E94E1126B017C01BB2039F00B561F4FB5
:100AF0000B52114010F4AA24A394229682E0C2362D
:100B0000D80749F6C092DA01D092DB01E092DC010D
:100B1000F092DD01AA2011F00E94B201E0908B0159
:100B2000F0908C0100918D0110918E01A801970128
:100B3000205D3740404050408091DE019091DF01C0
:100B4000A091E001B091E10182179307A407B507D6
:100B500040F580EDE81687E0F80680E0080780E0C1
:100B60001807F8F080917601882359F00E943C0222
:100B70000E943C02909581959F4F9093E301809352
:100B8000E20180918B0190918C01A0918D01B09137
:100B90008E018093DE019093DF01A093E001B0937A
:100BA000E10180916D02882349F180918B01909140
:100BB0008C01A0918D01B0918E01885E9340A04080
:100BC000B04020916E0230916F02409170025091BE
:100BD0007102281739074A075B0780F48091D90111
:100BE000882361F080916502882341F081E593E0DC
:100BF0006FE471E00E9464100E94B20180916A0269
:100C0000882399F010926A0280916502882369F026
:100C100080916D02882349F080916B0290916C0263
:100C20000197029710F40E94B20120919301309134
:100C3000940140919501509196012115310541058E
:100C40005105B9F080918B0190918C01A0918D019B
:100C5000B0918E01281739074A075B0750F40E94AC
:100C60000E0110929301109294011092950110922E
:100C7000960181E593E00E94E01120918B01309173
:100C80008C0140918D0150918E01181619065CF46B
:100C900020938F01309390014093910150939201E2
:100CA0000E94B80423C020513742404050408091F8
:100CB0008F0190919001A0919101B09192018217C2
:100CC0009307A407B50790F40E94690280918B01F5
:100CD00090918C01A0918D01B0918E0180938F0134
:100CE00090939001A0939101B0939201DF91CF91E5
:100CF0001F910F91FF90EF90DF90CF90BF90AF903A
:100D00009F908F900895CF93DF938FEB92E060E0F8
:100D100070E00E940B0CC82FD0E0CE014E978734B4
:100D2000910548F08FEB92E060E070E046E40E94AD
:100D3000120CC6E4D0E088E891E06AE070E00E941E
:100D4000460B88E891E0BE010E945F0A64EF71E003
:100D500080E090E00E94D40C88E891E00E94F309C2
:100D600083E061E00E94680D8BE061E00E94680D05
:100D700082E061E00E94680D84E061E00E94680DFD
:100D800087E061E00E94680D88E061E00E94680DE4
:100D900089E061E00E94680D86E061E00E94680DD4
:100DA0008CE061E00E94680D8EE060E00E94680DBA
:100DB0008091B10087608093B10085B5887F8160A4
:100DC00085BD83E060E070E00E941E0C8BE060E077
:100DD00070E00E941E0C82E061E00E94A70D84E09A
:100DE00060E00E94A70D87E061E00E94A70D88E007
:100DF00060E00E94A70D87E792E00E94590787E70D
:100E000092E061E00E946A0787E792E068E570E09F
:100E100040E050E02CEC30E00E94D60987E792E0F9
:100E200068E570E041E050E020E230E00E94D60941
:100E300087E792E068E570E042E050E023E130E0CF
:100E40000E94D60987E792E068E570E043E150E050
:100E500020E230E00E94D60987E792E068E570E082
:100E600048E150E024E530E00E94D60987E792E0AF
:100E700068E570E047E150E02EE330E00E94D609DB
:100E8000F89482E08093680081E080936C0078940D
:100E900081E593E040E052EC61E070E00E9459117E
:100EA00081E593E060E671E00E946410DF91CF91EC
:100EB0000895449A459AE9EBF0E080818E7F808323
:100EC00080818D7F808388E48093B80084E4809360
:100ED000BC000895662311F488E401C08CE080937F
:100EE000B8000895FC018091720290917402981BE1
:100EF00090937302882319F410927302089581501D
:100F000080937202E90FF11D828108950895EF9296
:100F1000FF920F931F930E94C60C7B018C0184E902
:100F20008093BC001BC021153105E1F00E94C60C66
:100F30006E197F09800B910B20917502309176021A
:100F400040E050E0621773078407950738F010926D
:100F5000BC0084E48093BC0081E009C0209175024C
:100F6000309176028091BC0084FDDDCF80E01F913E
:100F70000F91FF90EF900895CF92DF92EF92FF9242
:100F80001F93162F0E94C60C6B017C01112311F0D8
:100F900084EC01C084E88093BC001BC0211531059E
:100FA000E1F00E94C60C6C197D098E099F09209101
:100FB00075023091760240E050E0621773078407B3
:100FC000950738F01092BC0084E48093BC0091E057
:100FD00019C020917502309176028091BC0087FF84
:100FE000DDCF8091B900887F883349F49091B900B2
:100FF000987F1092BC0084E48093BC0003C0909161
:10100000B900987F892F1F91FF90EF90DF90CF90CC
:101010000895EF92FF920F931F93CF93DF93EC010C
:101020006093BB000E94C60C7B018C0184E8809316
:10103000BC001BC021153105E1F00E94C60C6E19E1
:101040007F09800B910B209175023091760240E070
:1010500050E0621773078407950738F01092BC00C0
:1010600084E48093BC0011E020C02091750230918F
:1010700076028091BC0087FFDDCF8091B900887F28
:10108000883211F410E011C01091B900187F8091DE
:10109000B900887F803321F4CE010E94870705C004
:1010A0001092BC0084E48093BC00812FDF91CF912B
:1010B0001F910F91FF90EF900895EF92FF920F9381
:1010C0001F93CF93DF93EC016093BB000E94C60C8B
:1010D0007B018C0184E88093BC001BC02115310585
:1010E000E1F00E94C60C6E197F09800B910B2091D4
:1010F00075023091760240E050E062177307840772
:10110000950738F01092BC0084E48093BC0011E095
:101110001DC020917502309176028091BC0087FF3E
:10112000DDCF8091B900887F883179F08091B90056
:10113000887F803499F409C08091B900887F883411
:10114000B1F4CE010E94870701C010E0812FDF912A
:10115000CF911F910F91FF90EF9008951091B900DA
:10116000187F8091B900887F803231F7EACF1092E2
:10117000BC0084E48093BC00E9CFEF92FF920F9310
:101180001F930E94C60C7B018C0184EA8093BC00F3
:101190001BC021153105E1F00E94C60C6E197F09B4
:1011A000800B910B209175023091760240E050E067
:1011B000621773078407950738F01092BC0084E427
:1011C0008093BC0091E021C020917502309176029D
:1011D0008091BC0087FFDDCF8091B900887F883087
:1011E00099F08091B900887F8031A9F40DC0909169
:1011F000B900987F1092BC0084E48093BC0005C0C5
:101200009091B900987F01C090E0892F1F910F91B4
:10121000FF90EF9008958091B900887F883381F71F
:10122000E6CFEF92FF920F931F93CF93DF93EC01E2
:10123000162F042FE22E10927202109273022223B4
:1012400011F4EE24E394EA94E982E3941882CE0147
:101250000E94BD088883882309F061C0110FCE0168
:10126000612F0E945D088883882329F0813009F06E
:1012700056C082E054C0CE01602F0E9409088883C6
:10128000882329F0813009F04AC083E048C0CE01AC
:101290000E94BD088883882329F0813009F03FC06F
:1012A00084E03DC01F5FCE01612F0E945D088883EE
:1012B000882319F48E01FF2425C0813081F585E053
:1012C0002EC08981F81651F4CE0160E00E94BC075F
:1012D0008883813019F1883551F021C0CE0161E059
:1012E0000E94BC0788838130C9F08035C1F48091A9
:1012F000BB00F8018283F394F0927202F0927402C0
:101300000F5F1F4FFE14E8F2CE010E94870788830B
:10131000882329F0813019F487E001C086E0DF914D
:10132000CF911F910F91FF90EF9008950E941109A6
:101330000895FF920F931F93CF93DF93EC01162F25
:10134000042FF22E18820E94BD088883882341F55D
:10135000110FCE01612F0E945D088883882321F040
:101360008130F1F482E01CC0CE01602F0E94090898
:101370008883882339F4CE016F2D0E940908888361
:10138000882319F0813061F40AC0CE010E948707DA
:101390008883882329F0813019F487E001C083E035
:1013A000DF91CF911F910F91FF9008950E949909AD
:1013B0000895FC01809199028C3090F480838F5FB6
:1013C00080939902815090E0FC01EE0FFF1FE80F1F
:1013D000F91FE656FD4F88EB9BE0928381830895C9
:1013E0008FEF80830895DC018C9190E0FC01EE0F7B
:1013F000FF1FE80FF91FE656FD4F80818F7B80832A
:101400008C916CE00E941E1590E0AC01440F551FBA
:10141000480F591F440F551F440F551F20E030E05F
:10142000C901840F951FFC01EE0FFF1FE80FF91F84
:10143000E656FD4F808186FD05C02F5F3F4F2C3063
:10144000310571F70895FC0120812C30B8F58181B8
:10145000992787FD909548E850E0481B590B440FA9
:10146000551F440F551F6417750784F08281992713
:1014700087FD909548E552E0481B590B440F551FD6
:10148000440F551F641775070CF4AB0142505040D0
:10149000CA01AA2797FDA095BA2F880F991FAA1FE6
:1014A000BB1F4FB7F89430E0F901EE0FFF1FE20FBA
:1014B000F31FE656FD4F928381834FBF0895AF928D
:1014C000BF92CF92DF92EF92FF920F931F93CF9331
:1014D000DF93EC019B0182E0603278070CF048C09A
:1014E00077FF03C020E030E005C0653B710514F0D4
:1014F00024EB30E000D000D0B901882777FD80953B
:10150000982F2981332727FD3095E8E8AE2EB12C9E
:10151000A21AB30AAA0CBB1CAA0CBB1CCC24B7FC95
:10152000C094DC2CEA81FF27E7FDF09528E532E046
:101530002E1B3F0B220F331F220F331F442737FD73
:101540004095542FEDB7FEB72183328343835483F4
:1015500020E030E040E050E004EBE02EF12C012DE3
:10156000112D0E9486109B010F900F900F900F90ED
:10157000CE01B9010E94230ADF91CF911F910F91F3
:10158000FF90EF90DF90CF90BF90AF900895CF92F3
:10159000DF92EF92FF921F93CF93DF93EC01162F10
:1015A0007A01690188818C3008F064C0862F61E07F
:1015B0000E94680D888190E0FC01EE0FFF1FE80F8C
:1015C000F91FE656FD4F1F738081807C812B80833D
:1015D00080E292E08E199F0964E070E00E942A1573
:1015E000698380E699E08C199D0964E070E00E94AF
:1015F0002A156A83A8818A2F6CE00E941E15682F25
:1016000070E0AB01440F551F460F571F440F551F85
:10161000440F551F20E030E0C901840F951FFC01E5
:10162000EE0FFF1FE80FF91FE656FD4F808186FD84
:1016300015C02F5F3F4F2C30310571F724C0109239
:10164000800082E0809381001092850010928400D7
:10165000B19A80916F00826080936F008A2F90E032
:10166000FC01EE0FFF1FE80FF91FE656FD4F8081CA
:10167000806480838881DF91CF911F91FF90EF90EC
:10168000DF90CF900895672BD1F2E8CF40E252E08F
:1016900020E639E00E94C70A08951F920F920FB604
:1016A0000F9211242F933F934F935F936F937F93E8
:1016B0008F939F93AF93BF93EF93FF938091BE025D
:1016C00087FF05C010928500109284002BC02091E6
:1016D000BE02332727FD30958091990290E02817AC
:1016E000390704F58091BE02992787FD9095FC018A
:1016F000EE0FFF1FE80FF91FE656FD4F808186FFB2
:1017000011C08091BE02992787FD9095FC01EE0FD4
:10171000FF1FE80FF91FE656FD4F80818F7360E0D1
:101720000E94A70D8091BE028F5F8093BE02209120
:10173000BE02332727FD30958091990290E028174B
:1017400039070CF04EC08091BE028C300CF049C0BD
:1017500020918400309185008091BE02992787FDF9
:101760009095FC01EE0FFF1FE80FF91FE656FD4FA5
:1017700081819281280F391F30938900209388003E
:101780008091BE02992787FD9095FC01EE0FFF1F07
:10179000E80FF91FE656FD4F808186FF2BC0809130
:1017A000BE02992787FD9095FC01EE0FFF1FE80F01
:1017B000F91FE656FD4F80818F7361E00E94A70DEF
:1017C00019C080E49CE905C0809184009091850057
:1017D000049690938900809388008FEF8093BE02D7
:1017E00009C08091840090918500049680549C49A2
:1017F00040F3EACFFF91EF91BF91AF919F918F910D
:101800007F916F915F914F913F912F910F900FBEFC
:101810000F901F901895F999FECF72BD61BDF89A8F
:1018200080B50895F999FECF1FBA72BD61BD40BD64
:101830000FB6F894FA9AF99A0FBE08951F93CF93B2
:10184000DF93182FEB0161E00E94680D209709F4E7
:101850004AC0CF3FD10509F449C0E12FF0E0E2557D
:10186000FF4F84918330C1F0843028F4813051F0EF
:101870008230B1F50CC0863019F1873049F18430DF
:1018800079F514C084B5806884BDC7BD33C084B504
:10189000806284BDC8BD2EC0809180008068809326
:1018A0008000D0938900C093880024C0809180007C
:1018B000806280938000D0938B00C0938A001AC00E
:1018C0008091B00080688093B000C093B30012C0D4
:1018D0008091B00080628093B000C093B4000AC0D1
:1018E000C038D1051CF4812F60E002C0812F61E077
:1018F0000E94A70DDF91CF911F9108951F920F9223
:101900000FB60F9211242F933F938F939F93AF9312
:10191000BF938091C4029091C502A091C602B0917C
:10192000C7023091C8020196A11DB11D232F2D5F62
:101930002D3720F02D570196A11DB11D2093C8020F
:101940008093C4029093C502A093C602B093C702CD
:101950008091C0029091C102A091C202B091C302D5
:101960000196A11DB11D8093C0029093C102A09366
:10197000C202B093C302BF91AF919F918F913F91EB
:101980002F910F900FBE0F901F9018958FB7F8945E
:101990002091C4023091C5024091C6025091C70205
:1019A0008FBFB901CA0108959B01AC017FB7F894BC
:1019B0008091C0029091C102A091C202B091C30275
:1019C00066B5A89B05C06F3F19F00196A11DB11D1A
:1019D0007FBFBA2FA92F982F8827860F911DA11D91
:1019E000B11D62E0880F991FAA1FBB1F6A95D1F72E
:1019F000BC012DC0FFB7F8948091C0029091C10244
:101A0000A091C202B091C302E6B5A89B05C0EF3F0A
:101A100019F00196A11DB11DFFBFBA2FA92F982F54
:101A200088278E0F911DA11DB11DE2E0880F991F1F
:101A3000AA1FBB1FEA95D1F7861B970B885E9340C0
:101A4000C8F2215030404040504068517C4F211531
:101A500031054105510571F60895789484B5826089
:101A600084BD84B5816084BD85B5826085BD85B542
:101A7000816085BDEEE6F0E0808181608083E1E8F1
:101A8000F0E0108280818260808380818160808329
:101A9000E0E8F0E0808181608083E1EBF0E080812C
:101AA00084608083E0EBF0E0808181608083EAE7FE
:101AB000F0E0808184608083808182608083808187
:101AC000816080838081806880831092C100089546
:101AD000CF93DF93482F50E0CA0186569F4FFC01F9
:101AE00034914A575F4FFA018491882369F190E05D
:101AF000880F991FFC01E859FF4FA591B491FC0193
:101B0000EE58FF4FC591D491662351F42FB7F89446
:101B10008C91932F909589238C93888189230BC076
:101B2000623061F42FB7F8948C91932F90958923AC
:101B30008C938881832B88832FBF06C09FB7F8942E
:101B40008C91832B8C939FBFDF91CF910895482F69
:101B500050E0CA0182559F4FFC012491CA0186566C
:101B60009F4FFC0194914A575F4FFA013491332300
:101B700009F440C0222351F1233071F0243028F4BD
:101B80002130A1F0223011F514C02630B1F02730F9
:101B9000C1F02430D9F404C0809180008F7703C055
:101BA000809180008F7D8093800010C084B58F77F6
:101BB00002C084B58F7D84BD09C08091B0008F774D
:101BC00003C08091B0008F7D8093B000E32FF0E0E0
:101BD000EE0FFF1FEE58FF4FA591B4912FB7F89469
:101BE000662321F48C919095892302C08C91892BD6
:101BF0008C932FBF0895682F70E0CB0182559F4FC3
:101C0000FC012491CB0186569F4FFC0144916A57F9
:101C10007F4FFB019491992319F420E030E03CC000
:101C2000222351F1233071F0243028F42130A1F027
:101C3000223011F514C02630B1F02730C1F0243025
:101C4000D9F404C0809180008F7703C08091800018
:101C50008F7D8093800010C084B58F7702C084B5DB
:101C60008F7D84BD09C08091B0008F7703C08091C3
:101C7000B0008F7D8093B000892F90E0880F991F6E
:101C800084589F4FFC01A591B4918C9120E030E0E5
:101C9000842311F021E030E0C9010895CF92DF9252
:101CA000EF92FF920F931F93CF93DF937C016B0111
:101CB0008A01C0E0D0E00FC0D6016D916D01D7015F
:101CC000ED91FC910190F081E02DC7010995C80FBD
:101CD000D91F015010400115110571F7CE01DF9198
:101CE000CF911F910F91FF90EF90DF90CF900895CB
:101CF000EF92FF920F931F938C01DC01ED91FC9109
:101D00000190F081E02D6DE009957C01D801ED9105
:101D1000FC910190F081E02DC8016AE009959C01D9
:101D20002E0D3F1DC9011F910F91FF90EF90089557
:101D3000CF93DF93EC016115710519F420E030E0D9
:101D40000FC0DB010D900020E9F71197A61BB70B20
:101D5000E881F9810280F381E02DAD0109959C01B4
:101D6000C901DF91CF9108954F925F927F928F9238
:101D70009F92AF92BF92CF92DF92EF92FF920F931A
:101D80001F93DF93CF93CDB7DEB7A1970FB6F8942B
:101D9000DEBF0FBECDBF2C01742ECB01223008F464
:101DA0002AE019A231E2C32ED12CCC0EDD1E822EE8
:101DB0009924AA24BB24672D752FA50194010E94A4
:101DC0003D1579018A01C801B701A50194010E945E
:101DD000FF14472D461B0894C108D1084A3014F45B
:101DE000405D01C0495CF6014083E114F104010546
:101DF000110521F07E2C5F2DC801DDCFC201B60197
:101E00000E94980EA1960FB6F894DEBF0FBECDBF0C
:101E1000CF91DF911F910F91FF90EF90DF90CF90C6
:101E2000BF90AF909F908F907F905F904F9008955C
:101E3000DC012115310541F4ED91FC910190F08117
:101E4000E02D642F099508950E94B40E0895CF9255
:101E5000DF92EF92FF920F931F93CF93DF93EC01EA
:101E60006A017B012115310541F4E881F981019076
:101E7000F081E02D642F09951FC02A303105D1F47F
:101E800077FF17C0E881F9810190F081E02D6DE2C4
:101E900009958C0144275527BA014C195D096E0933
:101EA0007F09CE012AE00E94B40E9801280F391F45
:101EB00004C02AE00E94B40E9C01C901DF91CF91B9
:101EC0001F910F91FF90EF90DF90CF900895EF92C8
:101ED000FF920F931F937B019A010027F7FC009557
:101EE000102FB801A7010E94270F1F910F91FF909B
:101EF000EF9008950E94980E08957F928F929F927E
:101F0000AF92BF92CF92DF92EF92FF920F931F9307
:101F1000CF93DF934C017A018B01722ECB01BA0172
:101F2000A80197010E94FB14882321F0C40168E6F0
:101F300071E021C0C0E0D0E057016801E894D7F813
:101F4000C601B5012FEF3FEF4FE75FE70E94FB149B
:101F5000882351F4C601B5012FEF3FEF4FE75FE74C
:101F60000E944513181614F0C1E0D0E0219739F013
:101F7000C4016CE671E00E94980EEC0193C0C801A8
:101F8000B7012FEF3FEF4FE75FE40E94941418165C
:101F900054F0C801B7012FEF3FEF4FE75FEC0E940D
:101FA0004513882324F4C40160E771E0E4CFC8013D
:101FB000B70120E030E040E050E00E94451387FD8B
:101FC00003C0C0E0D0E00EC0D401ED91FC910190BF
:101FD000F081E02DC4016DE20995EC0117FB10952D
:101FE00017F9109520E030E040E05FE3DD240BC0FE
:101FF000CA01B90120E030E040E251E40E944913F7
:102000009B01AC01D394D71498F3C801B7010E9487
:10201000E1125B016C010E94B6137B018C01C401CB
:10202000B801A7012AE030E00E94180FC80FD91F9D
:10203000772039F0C40164E771E00E94980EC80F60
:10204000D91FC801B7010E94E2139B01AC01C60170
:10205000B5010E94E01224C020E030E040E251E4EB
:102060000E9498147B018C010E94B1135B016C01EA
:10207000CC24B7FCC094DC2CC401B601A5012AE035
:1020800030E00E94270FC80FD91FC601B5010E947A
:10209000E4139B01AC01C801B7010E94E0127A94DD
:1020A0007720D1F6CE01DF91CF911F910F91FF9054
:1020B000EF90DF90CF90BF90AF909F908F907F90E8
:1020C00008950E947D0F0895EF92FF920F931F9342
:1020D0007C010E94980E8C01C7010E94780E080FA7
:1020E000191FC8011F910F91FF90EF900895CF9392
:1020F000DF930E942D0D0E948306CBE0D1E10E9468
:10210000E2042097E1F30E940B11F9CF2F923F9246
:102110004F925F926F927F928F929F92AF92BF92F7
:10212000CF92DF92EF92FF920F931F93DF93CF93A3
:10213000CDB7DEB73B014C0119012A016D897E89BB
:102140008F89988D6A197B098C099D09621A730A17
:10215000840A950AA40193010E94FF14E218F3086F
:1021600004091509A80197010E945F152A0D3B1D5E
:102170004C1D5D1DB901CA01CF91DF911F910F91D7
:10218000FF90EF90DF90CF90BF90AF909F908F9097
:102190007F906F905F904F903F902F90089508959B
:1021A0001F920F920FB60F9211242F933F934F93CC
:1021B0008F939F93EF93FF938091C00082FD1DC08A
:1021C0004091C6002091090330910A032F5F3F4FD1
:1021D0002F73307080910B0390910C0328173907EF
:1021E00071F0E0910903F0910A03E753FD4F40833A
:1021F00030930A032093090302C08091C600FF9127
:10220000EF919F918F914F913F912F910F900FBE22
:102210000F901F901895E0915D03F0915E03E05CD4
:10222000FF4F8191919120813181821B930B8F739C
:102230009070892B11F00E94CF1008951F920F9279
:102240000FB60F9211242F933F938F939F93EF9389
:10225000FF9320914D0330914E0380914F03909155
:1022600050032817390731F48091C1008F7D809386
:10227000C10014C0E0914F03F0915003E35FFC4FA5
:10228000208180914F039091500301968F7390703D
:102290009093500380934F032093C600FF91EF91DA
:1022A0009F918F913F912F910F900FBE0F901F9094
:1022B0001895AF92BF92DF92EF92FF920F931F9308
:1022C000CF93DF93EC017A018B01DD24403081EE66
:1022D000580780E0680780E0780711F0DD24D39488
:1022E00091E0A92EB12CEC89FD89DD2069F0C501B2
:1022F00008A002C0880F991F0A94E2F7808360E06B
:1023000079E08DE390E005C0108260E874E88EE12A
:1023100090E0A80197010E943D15215030404040B7
:102320005040569547953795279580E120303807DE
:1023300020F0DD2011F0DD24D6CFE889F989308343
:10234000EA89FB89208319A2EE89FF89408121E077
:1023500030E0C9010C8C02C0880F991F0A94E2F783
:10236000482B4083EE89FF894081C9010D8C02C052
:10237000880F991F0A94E2F7482B4083EE89FF8962
:102380004081C9010E8C02C0880F991F0A94E2F7A0
:10239000482B4083EE89FF8980810F8C02C0220F79
:1023A000331F0A94E2F7209528232083DF91CF91F1
:1023B0001F910F91FF90EF90DF90BF90AF90089525
:1023C000DC011C96ED91FC911D97E05CFF4F219183
:1023D000319180819181281B390B2F733070C90195
:1023E0000895DC011C96ED91FC911D97E05CFF4F78
:1023F00020813181E054F040DF01AE5BBF4F8D9111
:102400009C9111972817390719F42FEF3FEF07C058
:102410008D919C91E80FF91F8081282F30E0C90130
:102420000895DC011C96ED91FC911D97E05CFF4F37
:1024300020813181E054F040DF01AE5BBF4F8D91D0
:102440009C9111972817390719F42FEF3FEF10C00F
:102450008D919C911197E80FF91F20818D919C918E
:10246000119701968F73907011969C938E9330E024
:10247000C9010895DC0191968C919197882339F0D8
:102480005496ED91FC915597808186FFF9CF9196F6
:102490001C920895CF93DF93EC01EE85FF85E05CFD
:1024A000FF4F20813181E054F0402F5F3F4F2F7369
:1024B0003070DF01AE5BBF4F8D919C911197281753
:1024C0003907D1F3E05CFF4F80819181E054F04007
:1024D000E80FF91F6083EE85FF85E05CFF4F3183D5
:1024E0002083EE89FF89208181E090E00F8C02C07B
:1024F000880F991F0A94E2F7282B208381E089A393
:10250000EC89FD8980818064808381E090E0DF91A7
:10251000CF910895109254031092530388EE93E0E4
:10252000A0E0B0E08093550390935603A093570327
:10253000B09358038BE791E090935203809351033B
:1025400089EC92E090935E0380935D038DE093E0CD
:102550009093600380935F0385EC90E09093620317
:102560008093610384EC90E0909364038093630311
:1025700080EC90E0909366038093650381EC90E09B
:10258000909368038093670382EC90E090936A03D2
:102590008093690386EC90E090936C0380936B03C7
:1025A00084E080936D0383E080936E0387E08093E3
:1025B0006F0385E08093700381E080937103089539
:1025C0005058BB27AA270ED075C166D130F06BD109
:1025D00020F031F49F3F11F41EF45BC10EF4E0953E
:1025E000E7FB51C1E92F77D180F3BA176207730770
:1025F0008407950718F071F49EF58FC10EF4E095ED
:102600000B2EBA2FA02D0B01B90190010C01CA01AC
:10261000A0011124FF27591B99F0593F50F4503E57
:1026200068F11A16F040A22F232F342F4427585F49
:10263000F3CF469537952795A795F0405395C9F761
:102640007EF41F16BA0B620B730B840BBAF0915019
:10265000A1F0FF0FBB1F661F771F881FC2F70EC0B8
:10266000BA0F621F731F841F48F48795779567958B
:10267000B795F7959E3F08F0B3CF9395880F08F074
:102680009927EE0F979587950895D9D008F481E0A2
:1026900008950CD00FC107D140F0FED030F021F4E6
:1026A0005F3F19F0F0C0511139C1F3C014D198F354
:1026B0009923C9F35523B1F3951B550BBB27AA27C3
:1026C00062177307840738F09F5F5F4F220F331F35
:1026D000441FAA1FA9F333D00E2E3AF0E0E830D001
:1026E00091505040E695001CCAF729D0FE2F27D004
:1026F000660F771F881FBB1F261737074807AB07D2
:10270000B0E809F0BB0B802DBF01FF2793585F4F46
:102710002AF09E3F510568F0B6C000C15F3FECF360
:10272000983EDCF3869577956795B795F7959F5F0B
:10273000C9F7880F911D9695879597F90895E1E05F
:10274000660F771F881FBB1F621773078407BA07BE
:1027500020F0621B730B840BBA0BEE1F88F7E09519
:10276000089504D06894B111D9C00895BCD088F000
:102770009F5790F0B92F9927B751A0F0D1F0660F6D
:10278000771F881F991F1AF0BA95C9F712C0B13088
:1027900081F0C3D0B1E00895C0C0672F782F88279B
:1027A000B85F39F0B93FCCF3869577956795B395C7
:1027B000D9F73EF490958095709561957F4F8F4F36
:1027C0009F4F0895E89409C097FB3EF4909580953B
:1027D000709561957F4F8F4F9F4F9923A9F0F92FE7
:1027E00096E9BB279395F695879577956795B79565
:1027F000F111F8CFFAF4BB0F11F460FF1BC06F5F4B
:102800007F4F8F4F9F4F16C0882311F096E911C05C
:10281000772321F09EE8872F762F05C0662371F07D
:1028200096E8862F70E060E02AF09A95660F771F91
:10283000881FDAF7880F9695879597F90895990F6D
:102840000008550FAA0BE0E8FEEF16161706E8077A
:10285000F907C0F012161306E407F50798F0621B9B
:10286000730B840B950B39F40A2661F0232B242B70
:10287000252B21F408950A2609F4A140A6958FEF8F
:10288000811D811D089597F99F6780E870E060E0E1
:1028900008959FEF80EC089500240A9416161706F9
:1028A00018060906089500240A9412161306140641
:1028B00005060895092E0394000C11F4882352F0A4
:1028C000BB0F40F4BF2B11F460FF04C06F5F7F4F5C
:1028D0008F4F9F4F089557FD9058440F551F59F043
:1028E0005F3F71F04795880F97FB991F61F09F3FFD
:1028F00079F087950895121613061406551FF2CF26
:102900004695F1DF08C0161617061806991FF1CF75
:1029100086957105610508940895E894BB2766279C
:102920007727CB0197F908958ADF08F48FEF089590
:102930000BD0C0CFB1DF28F0B6DF18F0952309F037
:10294000A2CFA7CF1124EACFC6DFA0F3959FD1F382
:10295000950F50E0551F629FF001729FBB27F00D4D
:10296000B11D639FAA27F00DB11DAA1F649F6627A2
:10297000B00DA11D661F829F2227B00DA11D621FF1
:10298000739FB00DA11D621F839FA00D611D221FAB
:10299000749F3327A00D611D231F849F600D211D8F
:1029A000822F762F6A2F11249F5750408AF0E1F032
:1029B00088234AF0EE0FFF1FBB1F661F771F881F7B
:1029C00091505040A9F79E3F510570F05CCFA6CFC3
:1029D0005F3FECF3983EDCF3869577956795B79566
:1029E000F795E7959F5FC1F7FE2B880F911D969590
:1029F000879597F9089523DF880B990B0895629FB7
:102A0000D001739FF001829FE00DF11D649FE00DE6
:102A1000F11D929FF00D839FF00D749FF00D659F47
:102A2000F00D9927729FB00DE11DF91F639FB00D46
:102A3000E11DF91FBD01CF0111240895991B79E013
:102A400004C0991F961708F0961B881F7A95C9F73E
:102A50008095089597FB092E07260AD077FD04D0AC
:102A600049D006D000201AF4709561957F4F0895E3
:102A7000F6F7909581959F4F0895A1E21A2EAA1B13
:102A8000BB1BFD010DC0AA1FBB1FEE1FFF1FA2171E
:102A9000B307E407F50720F0A21BB30BE40BF50B1B
:102AA000661F771F881F991F1A9469F760957095A4
:102AB000809590959B01AC01BD01CF01089597FBD6
:102AC000092E05260ED057FD04D0D7DF0AD0001CF2
:102AD00038F450954095309521953F4F4F4F5F4FBB
:102AE0000895F6F790958095709561957F4F8F4F7B
:102AF0009F4F0895AA1BBB1B51E107C0AA1FBB1F14
:102B0000A617B70710F0A61BB70B881F991F5A9579
:102B1000A9F780959095BC01CD010895EE0FFF1F98
:0C2B20000590F491E02D0994F894FFCF8B
:102B2C003C76657273696F6E3A302E3132383E00E6
:102B3C003C6D6F766564200020003E003C73746F22
:102B4C00703E003C69643A3A6D616C673E00003C33
:102B5C00656570726F6D206572617365643E003CD3
:102B6C00686F72697A5F656570726F6D3A20003CB0
:102B7C0073746F706465746563746661696C3E0030
:102B8C003C72657365743E006E616E00696E660022
:102B9C006F7666002E0001000000004A124E0EE017
:082BAC00111112F1113A12009F
:00000001FF
